:1000000000308A00842900000A108A100A11820731
:1000100028340C34013406340A108A100A1182077D
:100020000C34413468346F346A3421340034303055
:100030008400000803192B280130A100A001A00BA7
:100040001F28A10B1E284A30A000A00B2528000065
:100050000000800B1C28003406080F39B400330E52
:10006000A000F030A0052008F03934048600061501
:1000700083160611000083120611831606118312DF
:100080000034B108031D46288610472886148316BD
:1000900086108312B20E3208B3002C20B20E320842
:1000A000B3002C200D30A000A00B542800341430D5
:1000B000B00017200F308316860583128610831632
:1000C000861083120611831606118312AA012A08CC
:1000D000023C031C73280230B00017200330B30029
:1000E0002C20AA0A67280D30A000A00B752802302A
:1000F000B3002C200D30A000A00B7C28AA012A08F8
:10010000023C031C8F282A080420AB00B1012B08F5
:10011000B20041200230B0001720AA0A7F288A11BD
:10012000C52901302D02AF002E08023C031D9A287C
:100130004030AF072F088038B000B1013008B2005E
:10014000412000342C08A0000C3020020319B528EF
:100150000A3020020319BD280D3020020319C328DC
:10016000083020020319C828CD28B1010130B2009F
:1001700041200230B0001720D9280130AD000230F4
:10018000AE009120D9280130AD00AE009120D928D1
:10019000B1011030B2004120D9282C081F3C031CAB
:1001A000D3280730AC050130B1002C08B200412043
:1001B000D92800342D08A1012C020318E2282C08AC
:1001C000A000EE28A0010830AE00AC0DA00D2D0857
:1001D00020020318A000A10DAE0BE52800342A0868
:1001E000A000AA1BF7282B1D01292030FC28A009FC
:1001F000A00A2008AA002D30A100AC00A2202B1DCF
:10020000AB152A08AC006430AD00DA202008AA0043
:1002100021083030031D13292B18AB15AB191929F0
:100220002B1A20301529AB112B12A1072108AC0085
:10023000A2202A08AC000A30AD00DA202008AA006B
:1002400021083030031D2829AB192C292B1A203006
:10025000A1072108AC00A2203030AA072A08AC0070
:10026000A220003430183629871137298715A511A7
:1002700025088316870053308312A000A00B3E2967
:10028000301C4429871145298715A5112508831697
:10029000870053308312A000A00B4C290034033098
:1002A000B00017200130B00032212D08B0003221FB
:1002B0000530AF00AF03031963292E08B0003221C7
:1002C0000310AE0C5A29A511250883168700831246
:1002D000871100342B082A07AC00AD010F30AE00A7
:1002E0004F210130AD002A08AE004F210130AD0092
:1002F0002B08AE004F210130AD002C08AE004F217D
:100300000A30B0001720003484011F308305073005
:1003100083169F00FF308312A500043083169F00D0
:1003200083121F08383901389F009412A51225083E
:1003300083168700831225162508831687008312EB
:10034000A5112508831687000030831294008316B8
:1003500094008312A001A01DB529073081018130CE
:1003600084000008C0390F388000640081308400A8
:100370000008C0392004800090010030A1009200E4
:1003800000308316920083125728AA012A080C20F5
:10039000AA0AAC00A22006302A02031DC629023098
:1003A000AA009630B0001720AA0BD1290030A10076
:1003B0001F08C73921049F000130AD00AE00912015
:1003C0001F151F19E1291E081E0EA8000F30A805D1
:1003D0005830AC00A2203A30AC00A2202030AC0053
:1003E000A2202808AA001830AB00EF200630AA008F
:1003F0002030AC00A220AA0BF8290830A1001F0869
:10040000C73921049F000130AD000230AE009120B9
:100410001F151F19092A1E081E0EA9000F30A90555
:100420005930AC00A2203A30AC00A2202030AC0001
:10043000A2202908AA001830AB00EF200630AA003D
:100440002030AC00A220AA0B202A0130AA002808E4
:10045000AB006A210230AA002908AB006A21D62924
:02046000630037
:02400E00F13F80
:00000001FF
